:100000005C2864001720031801282220A80108306A
:10001000A300232017200318A80AAB1EA801A20CD6
:10002000A30B0928AB1AA2132320220808003A08C0
:100030008400380884178004841300052B1B3806BD
:10004000FF3E080037172B081F39003EA1002A0881
:100050000E3E0318A10A371F40283713A0000230B4
:1000600052204028A301A200FF30A207031CA307CF
:10007000031C57280330A100E73040203428A10199
:10008000FC3EA000A109031C4B28FF300000A00784
:1000900003184628A0076400A10F45280800031094
:1000A000A10CA00CFF3E03184F28200857288313EB
:1000B000031383126400080007309F006400851C4E
:1000C000AC286400851C652861280130A300F43049
:1000D00033206400851C6E28BD017A29051583161E
:1000E000051105308312BA000130B8005430AA005F
:1000F0004030AB0001203A3C031D7A2801202A3C05
:10010000031D7A2801203D3C031D7A2801204A3C2A
:10011000031D7A2801203D3C031D7A280120313C33
:10012000031D7A280120653C031D7A280120BC00AC
:10013000831601309B0083123C0883169A0004301A
:100140009C0055309D00AA309D009C149C01831298
:100150000511831605118312831601309B000130AF
:100160009C0001308312322083161A088312BC00CF
:1001700085158316851183120530BA000130B80049
:100180005430AA004030AB000120413C031DC4287C
:100190000120643C031DC42801202B3C031DC428FE
:1001A00001202B3C031DC4280120543C031DC428FE
:1001B00001207E3C031DC4280120213C031DC428CE
:1001C0000120C100BE0164003E084102031C7929E0
:1001D0000530BA000130B8005430AA004030AB00FE
:1001E0000120C00064003E083C02031D7729640022
:1001F00080304002031C03298030C002861783161A
:1002000086138312072986138316861383126400CC
:1002100040304002031C13294030C00206178316E9
:10022000061383121729061383160613831264001C
:1002300020304002031C23292030C002861683167A
:10024000861283122729861283168612831264006F
:1002500010304002031C33291030C00206168316EA
:1002600006128312372906128316061283126400BF
:1002700008304002031C43290830C002861583164B
:100280008611831247298611831686118312640012
:1002900004304002031C53290430C00206158316A3
:1002A0000611831257290611831606118312640062
:1002B00002304002031C63290230C00286148316F8
:1002C00086108312672986108316861083126400B5
:1002D00001304002031C7229C00306148316061065
:1002E000831276290610831606108312BC28BE0FCF
:1002F000E328BC286400851C7E297A2964003D0817
:100300000C3C031D8429BD0164003D08003C031D15
:10031000A9290610831606108312861083168610EC
:100320008312061183160611831286118316861115
:100330008312061283160612831286128316861201
:1003400083120613831606138312861383168613ED
:10035000831264003D08013C031DB2290614831674
:100360000610831264003D08023C031DBF290610DD
:100370008316061083128614831686108312640077
:100380003D08033C031DCC2986108316861083127A
:10039000061583160611831264003D08043C031DF4
:1003A000D929061183160611831286158316861124
:1003B000831264003D08053C031DE629861183165F
:1003C00086118312061683160612831264003D08F6
:1003D000063C031DF32906128316061283128616A5
:1003E00083168612831264003D08073C031D002A11
:1003F000861283168612831206178316061383123B
:1004000064003D08083C031D0D2A061383160613DD
:100410008312861783168613831264003D08093CF5
:10042000031D322A061483160610831286148316BF
:1004300086108312061583160611831286158316FD
:1004400086118312061683160612831286168316E9
:1004500086128312061783160613831286178316D5
:1004600086138312051583160511831285158316CD
:100470008511640083123D080A3C031D5F2A0610A3
:1004800083160610831286108316861083120611B7
:1004900083160611831286118316861183120612A3
:1004A000831606128312861283168612831206138F
:1004B0008316061383128613831686138312640031
:1004C0003D080B3C031D842A061483160610831274
:1004D0008610831686108312061583160611831262
:1004E000861183168611831206168316061283124E
:1004F000861283168612831206178316061383123A
:1005000086138316861383120130BF0064001A30ED
:100510003F020318942A0A3032206400851C922A74
:10052000BD0A7A29BF0F862A051183160511831289
:10053000851183168511640083123D080A3C031D52
:10054000C12A061483160610831286148316861099
:1005500083120615831606118312861583168611DB
:1005600083120616831606128312861683168612C7
:1005700083120617831606138312861783168613B3
:10058000831264003D080B3C031DE62A0610831607
:1005900006108312861483168610831206118316A2
:1005A000061183128615831686118312061283168E
:1005B000061283128616831686128312061383167A
:1005C0000613831286178316861383120130BF0029
:1005D00064001A303F020318F62A0A303220640001
:1005E000851CF42ABD0A7A29BF0FE82A7A296300FC
:0205F000F72AE8
:02400E00463F2B
:024202000000BA
:00000001FF
